:100000000C944900189518951895189518951895F9
:100010001895189518951895189518951895189578
:100020001895189518951895189518951895189568
:100030001895189518951895189518951895189558
:100040001895189518951895189518951895189548
:10005000189518958A930FEF01BB80E882BB09D0F1
:10006000082F42E00E945700802F8823B9F780E8CC
:10007000F5CF192F282F80E090E001C001968F3F27
:100080000FEF9007D8F3822F912F089500008895E5
:10009000FECF0FE90DBF00E00EBFC0E8D0E00E9428
:1000A00065000E942A000E9446000C94460000242D
:1000B000E8E0EA9532F0001F001C0416D0F3041AA1
:0E00C000F8CF001F402D0095089501E008952F
:00000001FF
:00000001FF
